S02B000062696E2F6F70656E626C745F64656D6F70726F675F6E75636C656F5F73746D33326631303372622EC3
S31508000000F8060020F50F0008E10F0008E10F0008C8
S31508000010E10F0008E10F0008E10F0008E10F0008F2
S31508000020E10F0008E10F0008E10F0008E10F0008E2
S31508000030E10F0008E10F0008E10F0008E10F0008D2
S31508000040E10F0008E10F0008E10F0008E10F0008C2
S31508000050E10F0008E10F0008E10F0008E10F0008B2
S31508000060E10F0008E10F0008E10F0008E10F0008A2
S31508000070E10F0008E10F0008E10F0008E10F000892
S31508000080E10F0008E10F0008E10F0008E10F000882
S31508000090E10F0008E10F0008E10F0008E10F000872
S315080000A0E10F0008E10F0008E10F0008E10F000862
S315080000B0E10F0008E10F0008E10F0008E10F000852
S315080000C0E10F0008E10F0008E10F0008E10F000842
S315080000D0E10F0008E10F0008E10F0008E10F000832
S315080000E0E10F0008E10F0008E10F0008E10F000822
S315080000F0E10F0008E10F0008E10F0008E10F000812
S31508000100E10F0008E10F0008E10F0008E10F000801
S31508000110E10F0008E10F0008E10F0008E10F0008F1
S31508000120E10F0008E10F0008E10F0008E10F0008E1
S31508000130E10F0008E10F0008E10F0008E10F0008D1
S31508000140E10F0008E10F0008E10F0008E10F0008C1
S3150800015000B583B00023009301934FF48053C4F293
S3150800016002031A6842F001021A6059680022CFF6A3
S31508000170FF020A405A601A6822F0847222F480321A
S315080001801A601A6822F480221A605A6822F4FE025B
S315080001905A604FF41F029A601A6842F480321A6055
S315080001A04FF48053C4F2020340F2DC52196801F49A
S315080001B000310191009901310091019911B9009915
S315080001C09142F3D14FF48053C4F202031B6813F42F
S315080001D0003F06D141F25400C0F60000732100F03A
S315080001E0FBFA4FF40053C4F202031A6842F01002F5
S315080001F01A601A6822F003021A601A6842F00202AC
S315080002001A604FF48053C4F202035A685A605A6857
S3150800021042F400525A605A6842F480625A605A6838
S3150800022022F47C125A605A6842F4E8125A601A6834
S3150800023042F080721A604FF48053C4F202031A68BF
S3150800024012F0007FFBD04FF48053C4F202035A68C1
S3150800025022F003025A605A6842F002025A604FF4CA
S315080002608053C4F202035A6802F00C02082AFAD133
S315080002704FF48053C4F20203DA6942F40032DA61B9
S315080002809A6942F005029A614FF40063C4F20103C9
S315080002901A6822F470621A601A6842F430621A60A8
S315080002A01A6822F470421A601A6842F480421A6088
S315080002B000F004F800F00EF8FCE700BF08B500F0FF
S315080002C087FA00F0CBFB00F0ABFB00F00DF800F06E
S315080002D06DFA08BD08B500F07DFA00F0DBFB00F00A
S315080002E00FF800F043FA08BD08B500F063F800F00F
S315080002F0D1FA40F20003C2F2000300221A7008BDC8
S3150800030008B540F20400C2F2000000F00DFB012817
S315080003100BD140F20003C2F2000300221A7040F229
S315080003200400C2F2000000F065F808BD704700BF7F
S3150800033008B540F20003C2F200031B7813B9C9B22C
S3150800034000F0BEFA00F04EF808BD00BF40F2000308
S31508000350C2F200031878022806D0032806D001281E
S315080003600CBF0820402070470020704700207047C7
S3150800037040F20003C2F200031878022806D00328C8
S3150800038006D001280CBF082040207047002070477F
S315080003900020704708B500F01BF808BD40F244037A
S315080003A0C2F20003FE22DA7018710222A3F8442072
S315080003B0704700BF40F24403C2F2000300221A70DD
S315080003C09A6483F84320A3F844209A705A707047B9
S315080003D040F24403C2F200031878003018BF012027
S315080003E0704700BF40F24403C2F20003002283F8BC
S315080003F04320704738B504460178FF291CD140F2DE
S315080004004404C2F200040023637001252570FF220C
S31508000410E270102222716371FFF798FFA071FFF74F
S31508000420A7FFE071FFF7A4FF000A20726572A572A4
S315080004300823A4F8443079E140F24403C2F20003E9
S315080004401B78012B40F09081C939352900F26B8160
S31508000450DFE811F0DB0069016901650169016901DD
S315080004605901FC0042012F0169016901690169010D
S31508000470690169016901690169016901690169011E
S31508000480690169016901690169016901690169010E
S3150800049069016901690169016901690169016901FE
S315080004A069016901690169017F005400360073001A
S315080004B0690169016901A1006901B900BD00CE00A1
S315080004C04578FFF743FF0138854203DD2220FFF711
S315080004D065FF2BE140F24405C2F20005281DA96C10
S315080004E0627800F09FF9FF23EB706278AB6C1344D7
S315080004F0AB6463780133A5F8443017E14578FFF714
S3150800050025FF0138854203DD2220FFF747FF0DE16D
S31508000510616840F24405C2F20005A964281D6278A4
S3150800052000F080F9FF23EB706278AB6C1344AB6480
S3150800053063780133A5F84430F8E040F24403C2F288
S315080005400003FF22DA7042689A640122A3F8442065
S31508000550ECE040F24403C2F20003FF22DA709B6C1F
S31508000560406840B11844002213F8011B0A44D2B26D
S315080005708342F9D100E0002240F24403C2F20003AC
S31508000580C3F8072001221A7100225A719A710822AB
S31508000590A3F84420CAE040F24403C2F20003FF2253
S315080005A0DA7041F25C02C0F600029A6400221A71FF
S315080005B05A719A710721D9711A725A729A72082257
S315080005C0A3F84420B2E00020FFF7E8FEAEE040F2D0
S315080005D04403C2F20003FF22DA7000221A71597826
S315080005E059719A71DA711A720622A3F844209DE0AD
S315080005F040F24403C2F2000300221A705A70FF2226
S31508000600DA700122A3F8442090E040F24403C2F2D3
S3150800061000039D6CFFF79AFE411E2846621C00F0F7
S3150800062003FA18B93120FFF7B9FE7FE040F2440417
S31508000630C2F20004FF23E370A56CFFF787FE013DB5
S315080006402844A0640123A4F844306FE04578FFF7F6
S315080006507DFE0238854203DD2220FFF79FFE65E016
S3150800066040F24403C2F20003FF22DA700122A3F823
S315080006704420617839B900F0E7F9002856D13120CD
S31508000680FFF78CFE52E040F24403C2F20003986C76
S31508000690A21C00F0C9F918B93120FFF77FFE45E022
S315080006A040F24403C2F2000361789A6C0A449A64E1
S315080006B03CE040F24404C2F20004FF23E370002544
S315080006C025716571FFF742FEA071E57125726572A5
S315080006D00723A4F8443029E040F24403C2F2000399
S315080006E0986C616800F0A4F918B93120FFF756FE36
S315080006F01CE040F24403C2F20003FF22DA70012232
S31508000700A3F8442012E000F075F840F24403C2F260
S315080007100003FF22DA700122A3F8442006E0312004
S31508000720FFF73CFE02E02020FFF738FE40F24403C4
S31508000730C2F2000393F84330012B02D11020FFF7D1
S315080007402DFE40F24403C2F20003B3F844100BB284
S31508000750002B09DD40F24400C2F20000012380F8B4
S3150800076043300330FFF7E4FD38BD00BF08B5FFF797
S3150800077011FE012819D040F29003C2F200031B783B
S31508000780012B12D100F098F940F29403C2F200034B
S315080007901B6803F5FA73984207D340F29003C2F236
S315080007A0000300221A7000F025F808BD08B540F2CB
S315080007B09003C2F2000301221A7000F07DF940F29C
S315080007C09403C2F200031860FFF7D0FF08BD00BF0C
S315080007D0704700BF704700BF08B540F29803C2F2E1
S315080007E00003186040F29C03C2F200031960FFF789
S315080007F0F1FFFCE708B500F01FF990B1FFF796FD89
S3150800080000F040F900F01CF920F0604020F07F006D
S315080008104EF60853CEF20003186000F011F943684B
S31508000820984708BD70B5561EB6B24AB14C1E0E445E
S31508000830451A14F8013F2B55FFF7CCFFB442F8D1FF
S3150800084070BD00BF10B54FF48843C4F200031B887F
S3150800085003F080039BB2B3B14FF48843C4F200039C
S3150800086098801B8803F080039BB273B94FF48844C1
S31508000870C4F20004FFF7AEFF238803F080039BB29F
S31508000880002BF7D003E0002010BD012010BD012089
S3150800089010BD00BF4FF48843C4F2000300221A813A
S315080008A09A811A829A821A8340F271221A819A8947
S315080008B092B242F4005242F00C029A81704700BF8D
S315080008C02DE9F04106460C46402906D941F2640056
S315080008D0C0F600009221FFF77FFF2046FFF7B2FF20
S315080008E0012806D041F26400C0F600009621FFF701
S315080008F073FF2546ACB1002441F26407C0F6000731
S315080009004FF09F08FFF766FF305DFFF79BFF012852
S3150800091003D038464146FFF75FFF0134A3B2AB4226
S31508000920F0D3BDE8F08100BF10B540F2E503C2F28E
S3150800093000031B785BBB4FF48843C4F200031B8893
S3150800094003F020039BB2002B56D04FF48843C4F221
S3150800095000039A8892B240F2A003C2F200031A700A
S3150800096012F0FF0F4AD000F0A7F840F2E803C2F2EF
S315080009700003186040F2E403C2F200030020187076
S3150800098040F2E503C2F2000301221A7010BD40F2DC
S31508000990E403C2F200031A784FF48843C4F2000352
S315080009A01B8803F020039BB263B34FF48843C4F259
S315080009B000039C8840F2A003C2F2000399184C7009
S315080009C00132D2B240F2E401C2F200010A701B7889
S315080009D0934215D11149FFF725FF40F2E503C2F20C
S315080009E0000300221A70012010BD40F2E503C2F28E
S315080009F000030020187010BD002010BD002010BD97
S31508000A00002010BD00F058F840F2E803C2F20003D7
S31508000A101B6864339842E8D8002010BDA100002066
S31508000A2008B500F05BF908BD08B500F065F908BD22
S31508000A3008B500F089F908BD08B500F071FA08BDD7
S31508000A4008B500F0C7FA08BD08B500F03DFA10B1C0
S31508000A5000F09AFA08BD002008BD00BF4EF2100348
S31508000A60CEF2000300221A6041F63F11C0F20101DE
S31508000A7059609A600521196040F2EC03C2F200033E
S31508000A801A6070474EF21003CEF2000300221A6075
S31508000A90704700BF4EF21003CEF200031B6813F432
S31508000AA0803F1FBF40F2EC03C2F200031A6801320E
S31508000AB018BF1A60704700BF08B5FFF7EBFF40F292
S31508000AC0EC03C2F20003186808BD00BF4FF40053D8
S31508000AD0C4F202031A6942F080021A61704700BF25
S31508000AE0F8B507460024254641F28806C0F60006F2
S31508000AF0FFF770FEA359BB420ED8311949680B445B
S31508000B009F4209D241F28803C0F6000305EB45026D
S31508000B1003EB8203187AF8BD01350C349C2CE7D117
S31508000B20FF20F8BD2DE9F84380460068FFF7D8FF97
S31508000B30FF285CD04FF40053C4F2020340F223129C
S31508000B40C4F267525A6048F6AB12CCF6EF525A60B6
S31508000B503422DA60DB6813F0010F04D0FFF7B6FF22
S31508000B600020BDE8F8834FF40053C4F202031A6963
S31508000B7042F001021A61002508F104094FF40054F5
S31508000B80C4F20204D8F80030EF1859F80560B2B27A
S31508000B90EA52E36813F0010F05D0FFF71BFEE3687E
S31508000BA013F0010FF9D1330C7B80E36813F0010FC2
S31508000BB005D0FFF70FFEE36813F0010FF9D13B6884
S31508000BC0B34204D10435B5F5007FDBD101E000243A
S31508000BD000E001244FF40053C4F202031A6922F01C
S31508000BE001021A61FFF772FF2046BDE8F88300206C
S31508000BF0BDE8F88338B504460D4640F2F003C2F264
S31508000C000003984209D04FF4C043C0F60003994246
S31508000C100BD0FFF787FF20B917E040F2F424C2F2A1
S31508000C200004C5F3080393B903E040F2F004C2F2E6
S31508000C30000423689D420CD0204640F8045B2946F0
S31508000C404FF40072FFF7EEFD03E0002038BD0020E8
S31508000C5038BD204638BD00BF2DE9F04106460C4692
S31508000C6017461D464FEA51284FEA48280368B3F14C
S31508000C70FF3F06D140F8048B41464FF40072FFF758
S31508000C80D1FD3368434505D030464146FFF7B2FFEC
S31508000C900646D0B13368E41A3444043408F50078BB
S31508000CA0FFF798FD331DE31AB3F5007F06D33046E8
S31508000CB04146FFF79FFF064650B1041D17F8013B52
S31508000CC004F8013B013DEBD105E00020BDE8F081C9
S31508000CD00020BDE8F0810120BDE8F08140F2F42350
S31508000CE0C2F200034FF0FF321A6040F2F003C2F27C
S31508000CF000031A60704700BF70B504460D461646D5
S31508000D00FFF7EEFEFF281BD0681E2044FFF7E8FE1B
S31508000D10FF2817D0620A4FF4C043C0F60003B3EBAE
S31508000D20422F07BF40F2F000C2F2000040F2F42062
S31508000D30C2F20000214632462B46FFF78DFF70BDF2
S31508000D40002070BD002070BD2DE9F84304460E460C
S31508000D50FFF7C6FE0546701E2044FFF7C1FE04468F
S31508000D60FF2D18BFFF2800F0AB80854200F29F8058
S31508000D70022D40F29F800F2800F29F804FF4005307
S31508000D80C4F2020340F22312C4F267525A6048F6CC
S31508000D90AB12CCF6EF525A603422DA60DB6813F0F5
S31508000DA0010F04D0FFF792FE0020BDE8F8834FF448
S31508000DB00053C4F202031A6942F002021A6141F2B0
S31508000DC08809C0F600094F460026FFF703FD3B7A5F
S31508000DD0AB4208D141F28803C0F6000306EB46028F
S31508000DE053F8227005E001360C370D2EEDD14FF081
S31508000DF0FF37C8460025FFF7EDFC98F80830A342F0
S31508000E0008D141F28803C0F6000305EB450253F802
S31508000E10228006E0013508F10C080D2DEBD14FF0C4
S31508000E20FF384E460025FFF7D5FC337AA34209D191
S31508000E3041F28803C0F6000305EB450203EB820383
S31508000E405B6804E001350C360D2DECD10023C7EBA9
S31508000E5008084344C3F38F23E3B1013B9EB201362E
S31508000E60B60200254FF40054C4F20204EB1963617C
S31508000E70236943F040032361E36813F0010F05D0AB
S31508000E80FFF7A8FCE36813F0010FF9D105F58065B3
S31508000E90B542EBD14FF40053C4F202031A6922F0AB
S31508000EA002021A61FFF712FE0120BDE8F88300204E
S31508000EB0BDE8F8830020BDE8F8830020BDE8F88384
S31508000EC00020BDE8F88300BF00B583B040F2F00308
S31508000ED0C2F200031B68B3F1FF3F08BF01201CD014
S31508000EE040F2F003C2F2000399685A681144DA68BE
S31508000EF011441A6911445A6911449A690A44D9690C
S31508000F0053185B4202AA42F8043D46F25010C0F656
S31508000F1000000421FFF7F0FEFFE703B05DF804FBCD
S31508000F2046F20402C0F600024FF4C043C0F60003BE
S31508000F3010681B68184446F20803C0F600031B68CD
S31508000F40184446F20C03C0F600031B68184446F220
S31508000F501003C0F600031B68184446F21403C0F6D3
S31508000F6000031B68184446F21803C0F600031B6802
S31508000F70184446F25013C0F600031B681844D0F113
S31508000F80010038BF0020704708B540F2F003C2F2EE
S31508000F9000031B68B3F1FF3F06D040F2F000C2F22F
S31508000FA00000FFF7BFFD88B140F2F423C2F2000348
S31508000FB01B68B3F1FF3F0BD040F2F420C2F20000E9
S31508000FC0FFF7B0FD003018BF012008BD002008BD9E
S31508000FD0012008BD4FF4C040C0F60000704700BFAE
S31508000FE008B541F22410C0F600003621FFF7F4FBDD
S31508000FF008BD00BF10B572B640F20002C2F2000288
S3150800100040F20103C2F200039A4210D2131D0E4C9D
S31508001010E41A24F0030404340023104641F2501164
S31508001020C0F600015A581A500433A342FAD10748A9
S3150800103007494FF000028842B8BF40F8042BFADB94
S31508001040FFF786F810BD00BF04000020040000204A
S31508001050F80400206D61696E2E6300004F70656E9E
S31508001060424C54002E2E2F2E2E2F2E2E2F536F75B8
S315080010707263652F41524D434D335F53544D33329E
S315080010802F756172742E630000600008002000004E
S315080010900300000000800008002000000400000093
S315080010A000A00008002000000500000000C000089D
S315080010B0002000000600000000E0000800200000F4
S315080010C007000000000001080020000008000000DA
S315080010D00020010800200000090000000040010867
S315080010E0002000000A00000000600108002000003F
S315080010F00B00000000800108002000000C00000022
S3150800110000A00108002000000D00000000C0010832
S31508001110002000000E00000000E00108002000008A
S315080011200F0000002E2E2F2E2E2F2E2E2F536F75CA
S315080011307263652F41524D434D335F53544D3332DD
S315080011402F4743432F766563746F72732E630000CF
S30608001150048C
S70508000000F2
